:020000040000FA
:1000000000008A0103280730990083160313910129
:1000100070308F000F1D0A2800308100FF309500DE
:100020000830870083120313871101309300920177
:100030009115203084008001840A841F1B289717A3
:10004000613096000030F200403EF300403EF40084
:10005000403EF5008316031387113C3053200030D7
:10006000871583120313950072084F2073084F20E1
:1000700074084F2075084F2000304F2000304F206B
:1000800000304F2000304F203A3053200A30F10723
:10009000031C2A28F20AF30AF40AF50A2A288C1CFF
:0E00A0004F2895000800F000F00B54280800CF
:02400E00E43399
:00000001FF
